:0600000002005B02372044
:03000B0002335D60
:030013000233664F
:03001B0002002BB5
:030023000235D6CD
:10002B0032416C636F726E204D634272696465205E
:10003B00496E632E20536372697074204F53202DC9
:10004B002056657273696F6E20362E353020202056
:10005B00C2AF75D0007581567A00122D8175B8101C
:10006B0075A813787FE4F6D8FD758DFD758BFD753E
:10007B008C88758A0875892175880475368875355D
:10008B00087598C07E007F409020007400F0A3DEBE
:10009B00FCDFFA75A0787800E2A29392E3F4F52CDA
:1000AB0075A0807800E2F4F52DC2951232FAD2AF2A
:1000BB00D28CD28E12212D9000001232D5FAA312BF
:1000CB0032D5FBA31232D5FCA31232D5B46000405B
:1000DB00027460FD4C6018A31232D5F540A31232A6
:1000EB00D5A31232D5F54E90000212210560179060
:1000FB003A76122CFB7537287455F599780000D891
:10010B00FDD2030201A474AAF599780000D8FDC2B0
:10011B0003903A87122CFB122CB975382890000FDC
:10012B001232D5A2E792091230E5754520754400CD
:10013B00754B00754A30854E4FE54E60569000204A
:10014B00A3A3D54FFB75A02E7800854E4F1232D549
:10015B00F2A3081232D5F2A308B8000205A0D54FBE
:10016B00EC854E4F85458285448312139EA3A312C3
:10017B0032D5540F854B82854A83F0A385824B85FC
:10018B00834A854582854483A3A385824585834421
:10019B00D54FD112318812308B7A00122D81D29C1F
:1001AB001232FA1201D01202273001F7C2012003DA
:1001BB00F2122FAE120C23120F6C1211031213C07A
:1001CB001213C680DE75D0089021007F5A7E03E0A3
:1001DB00F5F0A3E0F8A3E0F9686034E5F0547FB4E0
:1001EB0000051202618028B401051204DD8020B4E1
:1001FB0002051202BE8018B40505120A718010B4F4
:10020B000905120B708008B408051205718000E512
:10021B00822406F5820FDEB775D00022300736E454
:10022B00B530130530122CB9903AE8122CFB903BE9
:10023B0011122D0D801F7405B530100530903B3A0F
:10024B00122CFB903B63122D0D800A745FB53005A9
:10025B000530122CD922AC83AD828F83898275D065
:10026B000075A0247800E0FB75F000E425F0F5F0B4
:10027B000582E5826508602DE0F208DBEF0582C59B
:10028B00F003547FB5F01E858209902400E0FBA398
:10029B00D20A753803121411300B03122FAE75D01E
:1002AB00088982800675373C75D008E5828C838D72
:1002BB0082F02285820C85830DE50FC3945A23248B
:1002CB005BF50B850F83850982E030E70FB4F800EF
:1002DB005007850B82758325F00204C3850B82754D
:1002EB008325E0B49000400EB4A0004053B4F0035B
:1002FB000203970204C3540FB540F8E50904B5088F
:10030B00030204D6850F83F582E030E7030204C3B2
:10031B001582E00509C3943CB408005020902400DA
:10032B00F5F0E540F0A37403F0A3E5F0F075D00011
:10033B007BFF902400D20A12141175D0080204C35B
:10034B00540FB540AEE50904B508030204D6850F7A
:10035B0083F582E030E7030204C360B41582E00545
:10036B0009C3943CB408005020902400F5F0E540FC
:10037B00F0A37402F0A3E5F0F075D0007BFF90249E
:10038B0000D20A12141175D0080204C3E508C395F4
:10039B0009B4090050030204AA850F83850982E082
:1003AB00B47F390582E0B47F028003B5402E05820D
:1003BB00E0B402280582E0B47F028008B41002800A
:1003CB0003B430180582E0B401028066B4060DE573
:1003DB0008C39509B40A0050060204AA0204950545
:1003EB0082E020E7F760F5B4210050F0F50B0582B1
:1003FB00E020E7E80582E020E7E2F5F00582E02067
:10040B00E7DA03548045F0F5F0858209902400E586
:10041B0040F0A37428F0A3E50B14F0A3E5F0F075FE
:10042B00D0007BFF902400D20A12141175D0080261
:10043B0004C30582E020E752C3943075F00AA4F59B
:10044B00F00582E020E743C3943025F075F00AA451
:10045B00F5F00582E020E732C3943025F0F5F00586
:10046B0082E0B4F725858209902400E540F0A3745F
:10047B0018F0A3E5F014F075D0007BFF902400D2A8
:10048B000A12141175D0080204C330E7030204BE2C
:10049B0075373C850B8275832574F7F00204C38591
:1004AB000F83850982E020E70A0582E582B508F50E
:1004BB000204D68582091509850C82850D83E50911
:1004CB0004F0F509650860030202CE850C82850DE8
:1004DB008322AC83AD8275D010E508B50903020504
:1004EB0066850F83850982E00509B4F5ECA809152B
:1004FB0009E508C398B405005003020566120A1AF1
:10050B00B54045902400F0A3F5F0120A1AFBB40392
:10051B0000503525F0F5F0120A1A602CB44000504B
:10052B0027F925F0F5F0E92405FAE508C39509FE4E
:10053B00B512004026120A1AF0A325F0F5F0D9F5F2
:10054B00120A1AB5F002800875373C05090204E45B
:10055B00753803120A2A88090204E475D008E509E4
:10056B008C838D82F022AC83AD8275D010E508B5FB
:10057B00090302063A850F83850982E0B4F10280F4
:10058B0004050980E88509F005F0E508B5F0087564
:10059B00D0088C838D8222850F8385F082E0B4F1A5
:1005AB000280DEB4F202800405F080DEE508B509B6
:1005BB000302063A850F83850982E00509B4F10F22
:1005CB0074011209D075A02078C8E4F20205B7B403
:1005DB00F2161209F730E00AC2E0C2E11209D002AA
:1005EB00064575373C0205B7F5F01209F720E00612
:1005FB0075373C0205B7F8E5F0B4F009E8D2E11223
:10060B0009D00205B7E830E10BC2E11209D0E5F0E1
:10061B0024F0F5F075A02078C8E275A03378002897
:10062B00F8E5F0F2E80475A02078C8F20205B7757A
:10063B00D008E5098C838D82F02275A02078C8E262
:10064B00B40300500675373C0206E375A0337800FF
:10065B0028F818E2F5F0790018E229F918B8FFF933
:10066B00E9B5F002800675373C0206E375A03378D6
:10067B00009020C412097B120910B4000675373C98
:10068B000206E3B40121E49020B4F0A3F0A3F0A39D
:10069B00F09020B8F0A3F0A3F0A3F09020BCF0A34F
:1006AB00F0A3F0A3F080129020B412097B9020B835
:1006BB0012097B9020BC12097B7900C0129020C8D4
:1006CB00E0FA1AE4F5F0E2F3080905F0EAB510F6E2
:1006DB00E5F0F0D0120206E602063A120910B40257
:1006EB00399020B4E0B4FF1AA3E0B4FF15A3E0B433
:1006FB00FF10A3E0B4FF0B1209F7D2E31209D002EB
:10070B0007257582B4E0700FA3E0700BA3E07007B0
:10071B00A3E0B5400280030207EE75A0337800908A
:10072B0020C012097B9020C0E0A3B40016E0A3B454
:10073B000011E0A3B4000CE0B404028009B4003B48
:10074B000207EB0207EBE2B4003108E22403FEE2FE
:10075B00FE08902400E540F0A3E2F008A3EEB510EC
:10076B00F890240075D000D20A7538031214117555
:10077B00D0101209F730E3090207EE75373C020778
:10078B00EB75A02078C4120938120910B402147545
:10079B00A02078B812093875A02078B412093874E3
:1007AB0005F0A3E4F0A37401F0A375A02078C8E2D0
:1007BB00F975A0337800E2F008A3E8B511F875A03D
:1007CB0024780075F000A982E20825F0F5F0E8B571
:1007DB0011F6E5F0F0A3E50FC3945AFA091208AE2F
:1007EB000208579020BCE0700EA3E0700AA3E070E3
:1007FB0006A3E07002805514F0B4FF187582BEE0BA
:10080B0014F0B4FF0F7582BDE014F0B4FF067582CF
:10081B00BCE014F0E50FC3945AF5F0902100E5828B
:10082B002408F5827A01E0547FB40816E5F0B5127E
:10083B0002800FAD82AE83AFF012085A8D828E8389
:10084B008FF0E5822408F5820ABA03DA0206E390F8
:10085B00240075A02078C412093875A02078B41232
:10086B00093875A02078B812093875A02078BC1209
:10087B00093875A02078C8E2F975A0337800E2F04A
:10088B0008A3E8B511F875A024780075F000A982CB
:10089B00E20825F0F5F0E8B511F6E5F0F0A3091242
:1008AB0008AE2290340074F1F0A375A0247800E216
:1008BB0008B4F007F0A3E4F0A3801CB4F10A74F0C1
:1008CB00F0A37401F0A3800FB4F20A74F0F0A374D8
:1008DB0002F0A38002F0A3E8B511D474F2F0A3A93F
:1008EB008290240075A0347800E2F008A3E582B56D
:1008FB0011F775D000902400AB11AA12D20A122D59
:10090B008B75D01022C082C0839020C4E0B4001637
:10091B00A3E0B40011A3E0B4000CA3E0B401028087
:10092B0007B4020280027400D083D08222E20860F6
:10093B001674FDF0A30808E218F0A3E218F0A3E286
:10094B0018F0A3E2F0A322E208601174FEF0A308F2
:10095B00E218F0A3E218F0A3E2F0A322E208600C85
:10096B0074FFF0A3E218F0A3E2F0A322E2F0A322BB
:10097B00C011E2F9B9FD1708080808E218F0A3E264
:10098B0018F0A3E218F0A3E2F00808088033B9FED0
:10099B0014E4F0A3080808E218F0A3E218F0A3E2AD
:1009AB00F00808801CB9FF10E4F0A3F0A30808E2DC
:1009BB0018F0A3E2F0088009E4F0A3F0A3F0A3E29F
:1009CB00F008D01122C009C082C083C0E0E50FC37C
:1009DB00945AF509902100E5822408D509FB2407D8
:1009EB00F582D0E0F0D083D082D00922C009C0823A
:1009FB00C083E50FC3945AF509902100E5822408C2
:100A0B00D509FB2407F582E0D083D082D00922C020
:100A1B0083C082850F838882E008D082D0832275C1
:100A2B00D0007BFF902400D20A121411E513B400FE
:100A3B0002802FB40214E50FC3945AFA850F8385F5
:100A4B000982E516FBD20A122D8BE50FC3945AFAD5
:100A5B0074AA3012027455902400F07B01D20A1252
:100A6B002D8B75D01022AC83AD8275D010A809E503
:100A7B0008C398B40C005003020B65850F83E5097E
:100A8B002402F582E0B43A028066B42D60A809E531
:100A9B0008C398B417005003020B65E5092416F53B
:100AAB0082E0B40D48902400A8097919120BC612E4
:100ABB000BF608791A120BC6120BF608791B120BE0
:100ACB00C6120BF6E82406F8791C120BC6120BF6AD
:100ADB0008791D120BC6120BF608791E120BC612E3
:100AEB000BF6791FE4120BF6E8F5098080020B6018
:100AFB00E509240BF582E0B40D5BA809E8F9120BAC
:100B0B00C6B41800504C120A1AB43A46120BC6B4AB
:100B1B003C00503E120A1AB43A38120BC6B43C00D1
:100B2B005030753803902400E9F8791C120BC6126B
:100B3B000BF608791D120BC6120BF608791E120B59
:100B4B00C6120BF6791FE4120BF6E509240CF50916
:100B5B00417875373C0509020A7875D008E5098C90
:100B6B00838D82F022AC83AD8275D010A809E50885
:100B7B00C398B405004039850F83850982E0B443DF
:100B8B002AA809E5092403F8E8120BC6601AB46316
:100B9B0000501514758330F582E0D2E2F0753803FE
:100BAB00E5092405F50980C475373C0509020B7767
:100BBB0075D008E5098C838D82F022C083C08285B5
:100BCB000F838882E0080582C39430B4060050146A
:100BDB0075F00AA4F5F0E008C39430B40A00500491
:100BEB0025F0800274FFD082D08322C0F0F5F0E5AF
:100BFB0040F0A37428F0A3E9F0A3E5F0F0A32428B8
:100C0B002903547FF075D0007BFF902400D20A1289
:100C1B00141175D010D0F022907800E0A29392E3DB
:100C2B00F4F8C52C6830E00CC0E0A26075F000123F
:100C3B000D22D0E030E10CC0E0A26175F001120D85
:100C4B0022D0E030E20CC0E0A26275F002120D225D
:100C5B00D0E030E30CC0E0A26375F003120D22D09C
:100C6B00E030E40CC0E0A26475F004120D22D0E079
:100C7B0030E50CC0E0A26575F005120D22D0E03016
:100C8B00E60CC0E0A26675F006120D22D0E030E74C
:100C9B0008A26775F007120D22908000E0F4F8C5EA
:100CAB002D6830E00CC0E0A26875F008120D22D060
:100CBB00E030E10CC0E0A26975F009120D22D0E022
:100CCB0030E20CC0E0A26A75F00A120D22D0E030BF
:100CDB00E30CC0E0A26B75F00B120D22D0E030E4F8
:100CEB000CC0E0A26C75F00C120D22D0E030E50CBC
:100CFB00C0E0A26D75F00D120D22D0E030E60CC0F5
:100D0B00E0A26E75F00E120D22D0E030E708A26F54
:100D1B0075F00F120D2222920590257DE0700302D3
:100D2B000E84F54F754D00754C26854D82854C8391
:100D3B00E0F9A3E0FAA3E0A3A385824D85834C8958
:100D4B00828A83F545C0F075F002A4F54B85F04A15
:100D5B00D0F0A3A31232D5FBA31232D5FCA31232CF
:100D6B00D5FDA31232D5FEA31232D5FFEF547FB5BA
:100D7B00F05EEB20E4052005578003300552EE6052
:100D8B000CB407005007120E8840028043903000CD
:100D9B00E5452582F582E030E23030E02FE54B244B
:100DAB0000F582E54A3431F5831213B1E582C39C19
:100DBB00E5839D5003020E81E545121E5975833064
:100DCB00854582E0D2E2F0020E81D2E2F0020E8182
:100DDB00A31232D5FEA31232D5FFEF547FB5F02B01
:100DEB00EB20E505200524800330051FEE600CB4D5
:100DFB0007005007120E8840028010903000E54526
:100E0B002582F582E0C2E2F0020E81A31232D5FEFA
:100E1B00A31232D5FFEF547FB5F02BEB20E6052064
:100E2B000524800330051FEE600CB4070050071239
:100E3B000E8840028010903000E5452582F582E057
:100E4B00D2E3F0020E81A31232D5FEA31232D5FFEC
:100E5B00EF547FB5F020EB20E70520051980033018
:100E6B000514EE600CB407005007120E8840028088
:100E7B0005E545121E59D54F0122020D35C082C022
:100E8B0083C0F0E5822407F582E5833400F58312F5
:100E9B0032D5F8A31232D5541F240BF975A025E3D4
:100EAB00F9EE30E708E8541F240BF8E2F8EE540F84
:100EBB002323900EC173020F0100020F0500020FD6
:100ECB001300020F2100020F3100020F4300020F2B
:100EDB005300020F0500020F1300020F2100020F37
:100EEB003100020F4300020F5300020F0100020FEB
:100EFB000100020F0100C3020F65E988F0B5F00491
:100F0B00D3020F65C3020F65E988F0B5F004C30285
:100F1B000F65D3020F65E988F0B5F0004004C302FA
:100F2B000F65D3020F65E988F0B5F0028006400427
:100F3B00C3020F65D3020F65E889F0B5F00040E2FC
:100F4B00C3020F65D3020F65E889F0B5F002800686
:100F5B004004C3020F65D3020F65D0F0D083D0825B
:100F6B0022200F0302109B90257EE0700302109B42
:100F7B00F54F754D00754C2A854D82854C83E0F9F4
:100F8B00A3E0FAA3E0A3A385824D85834C89828AD3
:100F9B0083F545C0F075F002A4F54B85F04AD0F00F
:100FAB00A3A31232D5FBA31232D5FCA31232D5FD6B
:100FBB00A31232D5FEA31232D5FFEE541FB4070095
:100FCB00404A12109E40028043903000E545258236
:100FDB00F582E030E23030E02FE54B2400F582E57E
:100FEB004A3431F5831213B1E582C39CE5839D50DE
:100FFB0003021087E545121E59758330854582E043
:10100B00D2E2F0021087D2E2F0021087A31232D59F
:10101B00FEA31232D5FFEE541FB407004017121077
:10102B009E40028010903000E5452582F582E0C29B
:10103B00E2F0021087A31232D5FEA31232D5FFEED7
:10104B00541FB40700401712109E400280109030BE
:10105B0000E5452582F582E0D2E3F0021087A3126A
:10106B0032D5FEA31232D5FFEE541FB40700400C4D
:10107B0012109E40028005E545121E59D54F030202
:10108B001090020F837E2090252B7400F0A3DEFCC2
:10109B00C20F22C082C083C0F0E5822407F582E52F
:1010AB00833400F5831232D5F8A31232D5541FF9CD
:1010BB0090252B2582F582E0C2046002D204EE302B
:1010CB00E719E8541FF890252B2582F582E0600282
:1010DB00D20475A025740B28F8E2F830041275A021
:1010EB0025740B29F9E3F9EE540F2323900EC173EA
:1010FB00C3D0F0D083D08222854E4FE54E700302D1
:10110B00135C754B00754A30754D00754C2E900075
:10111B0020E54E1213638582478583467543007520
:10112B004231754520754400854B82854A83E0200A
:10113B00E2030212F290001C1232D5540170089097
:10114B00001B1232D5603285458285448312139E73
:10115B0074152582F58274003583F5831232D530F0
:10116B00E017C082C08320E10474008002740190F8
:10117B003504F0D083D0828011C082C0837400907C
:10118B003504F0D083D08202126BA31232D5F8A3B0
:10119B001232D5F9A31232D5FA903502E0FB903515
:1011AB0001E0FC903500E0FDC3EB98F582EC99F57E
:1011BB00838542A0A843E582F208E583F2ED9A30DD
:1011CB00E7030212597071903505854FF0C3E58224
:1011DB0025F0F582E5833400F583E020E211E2701F
:1011EB001718E275F005B5F00280044002800990F3
:1011FB003503E07003021281903504E07003021294
:10120B00B285478285468312139E85824985834822
:10121B0012139EE5824583601F121376600A85497F
:10122B0082854883A3A380E2854D82854C83E54963
:10123B00F0A3E548F00212E5903504E06069854DB6
:10124B0082854C83E549F0A3E548F00212E585471A
:10125B008285468312139E8582498583480212E557
:10126B008543828542831213B1A38542A0A843E52F
:10127B0082F208E583F2854D82854C831213B1858A
:10128B00824985834812139EE582458360191213A8
:10129B00766047A3A3C20A12141120063D8549822A
:1012AB00854883A3A380D8903504E0702D854782B1
:1012BB0085468312139E8582498583488542A0A863
:1012CB00437400F208F2854B82854A83E030E105D6
:1012DB0010E3028002C2E2C2E4F0854D82854C83AA
:1012EB00E549F0A3E548F0854B82854A83E0F99008
:1012FB003505854FF0C3E58225F0F582E583340093
:10130B00F583E9F0D54F028048854B82854A83A34C
:10131B0085824B85834A854D82854C83A3A3858229
:10132B004D85834C854782854683A3A3858247855C
:10133B008346854382854283A3A38582438583426B
:10134B00854582854483A3A3858245858344021109
:10135B00339035037400F022C0F075F002A425829F
:10136B00F582E5F03583F583D0F022AD82AE8312A2
:10137B00139EAB82AC838543828542831213B1E506
:10138B0082C39BE5839C400474FF800274008D82B2
:10139B008E8322C0F01232D5F5F0A31232D5F5832D
:1013AB0085F082D0F022C0F0E0F5F0A3E0F5838564
:1013BB00F082D0F022AA24122D8122301347E5505F
:1013CB00B4024214F550780075A02574FFF208E5BD
:1013DB0040F2087400F208E52CF208E52DF208E55E
:1013EB002EF208E52FF208907000E0F208A3A3E0BC
:1013FB00F208A3A3E0F208E4F208F29025007A00C9
:10140B007B2B122D8B22C206AD82AE837A00123259
:10141B00E1FFA31232E1C212B467004003D21222E1
:10142B0090396275F002A42582F582E5F03583F5DB
:10143B0083E493F5F0A3E49385F083F582E47312D0
:10144B0015F60215F11216380215F112167902155E
:10145B00F11216B90215F11216FF0215F11217410E
:10146B000215F11217500215F112178F0215F11216
:10147B0017A70215F11217BF0215F11217E8021583
:10148B00F112193F0215F11230530215F112199D89
:10149B000215F11219E40215F1121B070215F112D4
:1014AB001C2A0215F1121C610215F1121CAD02155A
:1014BB00F1121CF90215F1121D530215F1121C3F0A
:1014CB000215F1121DAD0215F1121E130215F112C8
:1014DB001E2C0215F1121E450215F1121F7A021570
:1014EB00F112208B0215F11222B30215F10215F144
:1014FB00122CB90215F1122CD90215F11223090283
:10150B0015F11223370215F11223E10215F1122402
:10151B00050215F11224310215F112245E0215F1A8
:10152B0012248F0215F11224BE0215F11224F102BE
:10153B0015F11225220215F112255C0215F1122567
:10154B00970215F11225D60215F11226130215F189
:10155B001226540215F11226930215F11226BA0225
:10156B0015F11226E30215F112270F0215F11227BE
:10157B00400215F11227730215F11227AA0215F179
:10158B001227DF0215F11228180215F112284F024B
:10159B0015F112288E0215F11228CF0215F112291E
:1015AB00140215F11229570215F112299E0215F199
:1015BB001229E30215F1122A120215F11223650208
:1015CB0015F112239B0215F1122A430215F1122A6F
:1015DB00CC0215F1122B020215F1122CA30215F1FC
:1015EB00122B410215F18D828E83228D828E83A365
:1015FB00A31232E120E6291220EBB900104224F4A9
:10160B00F5F0902040E055F0F05228801FB9011002
:10161B004225F4F5F0902041E055F0F05229800C72
:10162B00543F2474F58275832074FFF0228D828ED3
:10163B0083A3A31232E120E6281220EBF4B9000FAA
:10164B005224F5F0902040E055F0F05228801EB95E
:10165B00010F5225F5F0902041E055F0F052298012
:10166B000C543F2474F5827583207400F0228D8214
:10167B008E83A3A31232E1F8541F232400C8122037
:10168B00EBFAA31232E175A020F208F2EAB9000DD1
:10169B00F5F0902040E045F0F042288010B9010DA4
:1016AB00F5F0902041E045F0F042298000228D8238
:1016BB008E83A3A31232E1F8541F232400C81220F7
:1016CB00EBFAA31232E175A020F208F2EAB900108E
:1016DB0042286224F4F5F0902040E055F0F080139E
:1016EB00B9011042296225F4F5F0902041E055F044
:1016FB00F08000228D828E83A3A31232E120E62993
:10170B001220EBB900106224F4F5F0902040E05564
:10171B00F0F05228801FB901106225F4F5F09020EB
:10172B0041E055F0F05229800C543F2474F582753A
:10173B008320E0F4F0228D828E83A3A31232E1FB8F
:10174B00A312218B22902200E0F8A3E0F5F075A004
:10175B005D902100E0547FB40105790102176C798B
:10176B0000903A32E993600BF20908E8B5F0F5D234
:10177B00068010902200E8C2ACF0200804D208D2F8
:10178B0099D2AC228D828E83A3A31232E1FAA312DB
:10179B0032E1FBA3122D8B6002D206228D828E8347
:1017AB00A3A31232E1FAA31232E1FBA3122E0660BD
:1017BB0002D206228D828E83A3A31232E1FA7B0121
:1017CB00A31232E190250B2582F582A20AC0D0D25A
:1017DB000A122D8BD0D0920A6002D206228D828EF5
:1017EB0083A3A31232E1FAA31232E1C0E0A31232B7
:1017FB00E1FF5407232390180573021824000218E5
:10180B005600021881000218A600021824000218C4
:10181B00240002182400021824D0E090250B258206
:10182B00F582E0780079007C00600F75F00A84A8DF
:10183B00F0600775F00A84A9F0FCE82430F8E9247D
:10184B0030F9EC2430FC7B030218C4D0E090250B5C
:10185B002582F582E0540F2430B43A00400224076D
:10186B00F9E054F0C42430B43A0040022407FC7869
:10187B00207B020218C4D0E090250B2582F582E074
:10188B0054072430F8E054380303032430F9E054B0
:10189B00C023232430FC7B030218C4D0E090250B1B
:1018AB002582F5827B01A20AC0D0D20A122D8BD0E1
:1018BB00D0920A607ED206807AEF5438039018CC0F
:1018CB00730218EB0002191F00021910000218F91D
:1018DB00000218EB000218EB000218EB000218EBE9
:1018EB00BB0102802FBC302CE9FCE8F9DBF2BC30E9
:1018FB0023E9FCE8F97820BB031ABC3017E9FCE8B4
:10190B00F97820800FBC300C7C20BB0307B9300466
:10191B0079208000902044ECF0A3E9F0A3E8F0904C
:10192B002044A20AC0D0D20A122D8BD0D0920A60CA
:10193B0002D206228D828E83A3A31232E1FAA31266
:10194B0032E1F8A31232E1F9A31232E190250B2513
:10195B0082F582E0FB9020447406F0A3E5404480BE
:10196B00F0FCA3E8F02CFCA37428F02CFCA3E9F00A
:10197B002CFCA3EBF02CA303547FF09020447B07AB
:10198B00A20AC0D0D20A122D8BD0D0920A6002D2FA
:10199B0006228D828E8375D010A3A31232E1FBA396
:1019AB00AD82AE83902100E5822408F5827A01E0B6
:1019BB00547FB40819A882A9838D828E8375D000B9
:1019CB00AA12AB13122D8B75D01088828983E582F6
:1019DB002408F5820ABA03D722854B82854A83E015
:1019EB00F98D828E83A3A31232E1FA232323FC7594
:1019FB00A021F8E920E442E2C2E7F2E408F208F29F
:101A0B00A31232E1FBA3122D8B75A021ECF8E2D2CD
:101A1B00E7F208080808081232E1F2A3081232E1D3
:101A2B00F2200606A3081232E1F2854B82854A8327
:101A3B00E0D2E4F0D206021B0608A31232E1240521
:101A4B002582F582E43583F5831232E1F5F0E2C3AA
:101A5B0095F0501E08080808E2F5F008E245F06022
:101A6B002D18E2C39401F2500408E214F2D20602DC
:101A7B001B06ABF0A3EA245AF5A078001232E1F56D
:101A8B00F0E2B5F009A308DBF3753803804A75A0C3
:101A9B0021EC2407F8E2600F14F28D828E83A3A34E
:101AAB00ECF8D206021A0275373C30092B90001461
:101ABB001232D5F8A31232D5F5838882E5822AF546
:101ACB0082E43583F5831232D5F8C3954E500975F0
:101ADB0083308882E0D2E2F075A021ECF8E2547FEB
:101AEB00B403028003B40704C2E78002D2E7F28595
:101AFB004B82854A83E0C2E4F0C20622854B828585
:101B0B004A83E0F98D828E83A3A31232E1FA232359
:101B1B0023FC75A021F8E920E442E2C2E7F2E408D5
:101B2B00F208F2A31232E1FBA3122E0675A021ECF0
:101B3B00F8E2D2E7F208080808081232E1F2A3082B
:101B4B001232E1F2200606A3081232E1F2854B8233
:101B5B00854A83E0D2E4F0D206021C2908A3123294
:101B6B00E124052582F582E43583F5831232E1F514
:101B7B00F0E2C395F0501E08080808E2F5F008E201
:101B8B0045F0602D18E2C39401F2500408E214F200
:101B9B00D206021C29ABF0A3EA245AF5A078001256
:101BAB0032E1F5F0E2B5F009A308DBF375380380F9
:101BBB004A75A021EC2407F8E2600F14F28D828E97
:101BCB0083A3A3ECF8D206021B2575373C30092BF7
:101BDB009000141232D5F8A31232D5F5838882E522
:101BEB00822AF582E43583F5831232D5F8C3954EFC
:101BFB0050097583308882E0D2E2F075A021ECF8B1
:101C0B00E2547FB403028003B40704C2E78002D21C
:101C1B00E7F2854B82854A83E0C2E4F0C206228D4F
:101C2B00828E83A3A31232E1547F232549F54950B9
:101C3B00020548228D828E83A3A31232E1FAA312EE
:101C4B0032E1F9EAC333FAE933F9EAC32549F54935
:101C5B00E93548F548228D828E83A3A31232E12009
:101C6B00E71810E60A1220EBB900047824801E2432
:101C7B0074F875A020E2701A8027547F1220EBB9FC
:101C8B000004782C8007B90104782D80005670026F
:101C9B00800FA31232E1547F232549F549500205E9
:101CAB0048228D828E83A3A31232E120E71810E61F
:101CBB000A1220EBB900047824801E2474F875A056
:101CCB0020E2601A8027547F1220EBB90004782C95
:101CDB008007B90104782D8000566002800FA31293
:101CEB0032E1547F232549F54950020548228D8264
:101CFB008E83A3A31232E120E71810E60A1220EB21
:101D0B00B900047824801E2474F875A020E2701AA0
:101D1B008035547F1220EBB90004782C8007B90171
:101D2B0004782D8000567002801DA31232E1FAA3B5
:101D3B001232E1F9EAC333FAE933F9EAC32549F57B
:101D4B0049E9FA3548F548228D828E83A3A31232D6
:101D5B00E120E71810E60A1220EBB9000478248082
:101D6B001E2474F875A020E2601A8035547F12206F
:101D7B00EBB90004782C8007B90104782D8000564C
:101D8B006002801DA31232E1FAA31232E1F9EAC319
:101D9B0033FAE933F9EAC32549F549E9FA3548F548
:101DAB0048228D828E83A3A31232E1F8C3954E5045
:101DBB00567583308882E030E24A30E04AC004C076
:101DCB0005900020E812136312139EA3A3A31232F3
:101DDB00D5FCA31232D5FDE8C0F075F002A42400A7
:101DEB00F582E5F03431F583D0F01213B1E582C3FF
:101DFB009CE5839DD005D004400DE8121E597583D8
:101E0B00308882E0D2E2F0228D828E83A3A312323D
:101E1B00E1F8C3954E50097583308882E0C2E2F039
:101E2B00228D828E83A3A31232E1F8C3954E500903
:101E3B007583308882E0D2E3F0228D828E83A3A358
:101E4B001232E1F8C3954E5004E8121E5922C0001D
:101E5B00C003C004C0F0F8900020E54E121363E8F5
:101E6B0012136312139EAB82AC8375832EE875F04D
:101E7B0002A4F582E5F03583F583EBF0A3ECF07566
:101E8B008331E875F002A4F582E5F03583F583E440
:101E9B00F0A3F07583308882E0C2E2C2E4F0C2E3C3
:101EAB00D0F0D004D003D00022902200E0F875A02F
:101EBB005D902100E0547FB400047402F20890009E
:101ECB00021232D5A3F2081232D5F208902200E8A2
:101EDB00C2ACF0200804D208D299D2AC22C004C004
:101EEB0005C00675A025784B7910750400750500A3
:101EFB0075060CD5041DD5051AD506177455C29B4E
:101F0B00C299F599750400750504D504FDD505FA3C
:101F1B0002005B3098DDE599F2C298EA70011B1A5A
:101F2B00EB7003EA601108D9C1784B7910E21232D9
:101F3B00C5A308D9F880AC7A007B20DAFEDBFC78ED
:101F4B004B7910E21232C5A308D9F8902100E05466
:101F5B007FB4011474AAC29BC299F59975040075DC
:101F6B000508D504FDD505FAD006D005D00422C24C
:101F7B00AF8D828E83A3A31232E1FAA31232E1FB5F
:101F8B00E599C29874AAC29BC299F5999000001268
:101F9B001EE802005B8D828E83A3A31232E1FAA3AB
:101FAB001232E1FB9000021232D5F8A31232D5C8DF
:101FBB0054F0241CC8500104F5838882745A1232E1
:101FCB00C5A374A51232C5A3EA1232C5A3EB123214
:101FDB00C5A3C000C001750000750100D500FDD57B
:101FEB0001FAD001D000C2AFE599C29874AAC29B86
:101FFB00C299F599121EE874AAC29BC299F59975FC
:10200B000400750504D504FDD505FA02005B201408
:10201B00FDC29BD214F599229000021232D5F8A37F
:10202B001232D5C854F0241CC8500104F5838882A1
:10203B001232D5B45A18A31232D5B4A511A3123249
:10204B00D5FAA31232D5FBA3BA000CBB0009E412DC
:10205B002019122019801AEA122019EB12201912DA
:10206B0032D5A31220191ABAFF011BBA00F1BB001B
:10207B00EE750400750504D504FDD505FA02005B69
:10208B009000021232D5FAA31232D5FB700CEA7013
:10209B0009E412201912201980278A828B83A3A3AB
:1020AB00AA82AB83EA122019EB12201990000012BE
:1020BB0032D5A31220191ABAFF011BBA00F1BB00CB
:1020CB00EE750400750504D504FDD505FA02005B19
:1020DB008D828E83A3A31232E1C2136002D213222C
:1020EB00F95407C90303035403C0E07401B9000298
:1020FB00800323D9FDF9D0E0C92278007900123290
:10210B00D528500109F8A3DC05BD00F28006BCFF01
:10211B00ED1D80EAE86A7007E96B7003E4800274D6
:10212B00FF2290000075A0987802E230E70BA3E540
:10213B0083B405F6C21102218AD2117A30122D1FF7
:10214B007A30122D1F7A38122D1F7A80122D1F7A9A
:10215B0006122D1F7A0C122D1F7A01122D1F7A4099
:10216B00122D1F7A5A122D3E7A40122D1F122D60FE
:10217B00B45AC1903A65122CFB903A4B122D0D229A
:10218B00EB60627A80122D1F1232E1B404005029E9
:10219B00A3DB028050B400047A808010B401047A6F
:1021AB00C08009B402047A9480027AD41232E1A37B
:1021BB00543F2AFA122D1F802AB40C08A37A01125D
:1021CB002D1F801FB40D03A38014B40A03A3800E2C
:1021DB00B40E2EDB11800EFA122D3EA380057AC0B1
:1021EB00122D1FDBA322A31232E114A3C082C083E2
:1021FB0090250B2582F582E0D083D08212226F804E
:10220B00E2B40FD3DB0280DDA31232E114A3C08250
:10221B00C08390250B2582F582E0D083D0821222D9
:10222B002E80C07C017A20C39464400C1C7A31C38D
:10223B0094644004C394640A2464C0E0122D3ED01D
:10224B00E07A31C3940A40030A80F81A240AC0E0EA
:10225B00BA3005EC60027A20122D3ED0E02430FA21
:10226B00122D3E227C017A20C39464400C1C7A31DF
:10227B00C394644004C394640A2464BA20028007A4
:10228B00C0E0122D3ED0E07A31C3940A40030A809D
:10229B00F81A240AC0E0BA3003EC7003122D3ED0BA
:1022AB00E02430FA122D3E228D828E83A3A31232AC
:1022BB00E15403FB7005903A988013B40105903AF2
:1022CB00A8800BB40205903AB88003903AC87A0103
:1022DB00122D1F7C10E493FA122D3EA3DCF77C1019
:1022EB007AC0122D1FEBC42474F582758320E06035
:1022FB00047A3180027A30122D3EA3DCF1228D82DA
:10230B008E83A3A31232E1FAA31232E1FBEA422439
:10231B00F4F5F0902040E055F0F05228EB4225F414
:10232B00F5F0902041E055F0F05229228D828E83FA
:10233B00A3A31232E1FAA31232E1FBEAF45224F521
:10234B00F0902040E055F0F05228EBF45225F5F0D8
:10235B00902041E055F0F05229228D828E83A3A369
:10236B001232E1FAA31232E1FBEA7011EBF524F41D
:10237B00F5F0902040E055F0F052288012B4010F98
:10238B00EBF525F4F5F0902041E055F0F0522922C1
:10239B008D828E83A3A31232E1FAA31232E1FBEA00
:1023AB00701875A025740B2BF8E52CF275A025740D
:1023BB002B2BF874FFF2D20F801BB4011875A025DC
:1023CB00740B2BF8E52DF275A025742B2BF874FFED
:1023DB00F2D20F8000228D828E83A3A31232E1549E
:1023EB001FF9240BF8A31232E175A025F275A02575
:1023FB00742B29F874FFF2D20F228D828E83A3A344
:10240B001232E1541FF9240BF875A025E2F5F0A365
:10241B001232E1B5F00FA31232E1547F232549F5B7
:10242B004950020548228D828E83A3A31232E154B8
:10243B001F240BF875A025E2F5F0A31232E1B5F0DD
:10244B0002800FA31232E1547F232549F549500234
:10245B000548228D828E83A3A31232E1541F240BD5
:10246B00F875A025E2F5F0A31232E1C5F0B5F00046
:10247B004002800FA31232E1547F232549F54950C6
:10248B00020548228D828E83A3A31232E1541F24AE
:10249B000BF875A025E2F5F0A31232E1B5F0004080
:1024AB0002800FA31232E1547F232549F5495002D4
:1024BB000548228D828E83A3A31232E1541F240B75
:1024CB00F875A025E2F5F0A31232E1C5F0B5F002E4
:1024DB0080044002800FA31232E1547F232549F57B
:1024EB004950020548228D828E83A3A31232E154F8
:1024FB001F240BF875A025E2F5F0A31232E1B5F01D
:10250B000280044002800FA31232E1547F2325493D
:10251B00F54950020548228D828E83A3A31232E126
:10252B00541FF9240BF875A025E2F5F0A31232E144
:10253B00B5F01DA31232E1FAA31232E1F9EAC3336B
:10254B00FAE933F9EAC32549F549E9FA3548F5487B
:10255B00228D828E83A3A31232E1541F240BF875B4
:10256B00A025E2F5F0A31232E1B5F002801DA31213
:10257B0032E1FAA31232E1F9EAC333FAE933F9EAA9
:10258B00C32549F549E9FA3548F548228D828E83F2
:10259B00A3A31232E1541F240BF875A025E2F5F02A
:1025AB00A31232E1C5F0B5F0004002801DA3123238
:1025BB00E1FAA31232E1F9EAC333FAE933F9EAC3D8
:1025CB002549F549E9FA3548F548228D828E83A3D2
:1025DB00A31232E1541F240BF875A025E2F5F0A3EA
:1025EB001232E1B5F0004002801DA31232E1FAA3D2
:1025FB001232E1F9EAC333FAE933F9EAC32549F5B3
:10260B0049E9FA3548F548228D828E83A3A312320D
:10261B00E1541F240BF875A025E2F5F0A31232E16B
:10262B00C5F0B5F00280044002801DA31232E1FA1E
:10263B00A31232E1F9EAC333FAE933F9EAC32549C4
:10264B00F549E9FA3548F548228D828E83A3A3120A
:10265B0032E1541F240BF875A025E2F5F0A31232DA
:10266B00E1B5F00280044002801DA31232E1FAA30F
:10267B001232E1F9EAC333FAE933F9EAC32549F532
:10268B0049E9FA3548F548228D828E83A3A312328D
:10269B00E1541FF9240BF875A025E2FAA31232E1DD
:1026AB002AF275A025742B29F974FFF3D20F228D12
:1026BB00828E83A3A31232E1541FF9240BF875A069
:1026CB0025E2FAA31232E1CAC39AF275A025742B44
:1026DB0029F974FFF3D20F228D828E83A3A31232BA
:1026EB00E1541FF5F0240BF8A31232E1541F240B15
:1026FB00F975A025E3F275A025742B25F0F874FF6E
:10270B00F2D20F228D828E83A3A31232E1541F24A7
:10271B000BF875A025E2F5F0A31232E1541F240B40
:10272B00F9E3B5F00FA31232E1547F232549F549A4
:10273B0050020548228D828E83A3A31232E1541FCF
:10274B00240BF875A025E2F5F0A31232E1541F24F7
:10275B000BF9E3B5F00280DCA31232E1547F2325A1
:10276B0049F54950020548228D828E83A3A312326C
:10277B00E1541F240BF875A025E2F5F0A31232E10A
:10278B00541F240BF9E3C5F0B5F0004002800FA3F2
:10279B001232E1547F232549F54950020548228D19
:1027AB00828E83A3A31232E1541F240BF875A0254C
:1027BB00E2F5F0A31232E1541F240BF9E3B5F0005C
:1027CB004002800FA31232E1547F232549F5495073
:1027DB00020548228D828E83A3A31232E1541F245B
:1027EB000BF875A025E2F5F0A31232E1541F240B70
:1027FB00F9E3C5F0B5F00280044002800FA312325A
:10280B00E1547F232549F54950020548228D828EDC
:10281B0083A3A31232E1541F240BF875A025E2F514
:10282B00F0A31232E1541F240BF9E3B5F00280043C
:10283B004002800FA31232E1547F232549F5495002
:10284B00020548228D828E83A3A31232E1541F24EA
:10285B000BF875A025E2F5F0A31232E1541F240BFF
:10286B00F9E3B5F01DA31232E1FAA31232E1F9EA52
:10287B00C333FAE933F9EAC32549F549E9FA35488F
:10288B00F548228D828E83A3A31232E1541F240BB1
:10289B00F875A025E2F5F0A31232E1541F240BF9D1
:1028AB00E3B5F00280DCA31232E1FAA31232E1F9B4
:1028BB00EAC333FAE933F9EAC32549F549E9FA35AD
:1028CB0048F548228D828E83A3A31232E1541F2434
:1028DB000BF875A025E2F5F0A31232E1541F240B7F
:1028EB00F9E3C5F0B5F0004002801DA31232E1FA06
:1028FB00A31232E1F9EAC333FAE933F9EAC3254902
:10290B00F549E9FA3548F548228D828E83A3A31247
:10291B0032E1541F240BF875A025E2F5F0A3123217
:10292B00E1541F240BF9E3B5F0004002801DA31204
:10293B0032E1FAA31232E1F9EAC333FAE933F9EAE5
:10294B00C32549F549E9FA3548F548228D828E832E
:10295B00A3A31232E1541F240BF875A025E2F5F066
:10296B00A31232E1541F240BF9E3C5F0B5F002803A
:10297B00044002801DA31232E1FAA31232E1F9EAFC
:10298B00C333FAE933F9EAC32549F549E9FA35487E
:10299B00F548228D828E83A3A31232E1541F240BA0
:1029AB00F875A025E2F5F0A31232E1541F240BF9C0
:1029BB00E3B5F00280044002801DA31232E1FAA3BA
:1029CB001232E1F9EAC333FAE933F9EAC32549F5DF
:1029DB0049E9FA3548F548228D828E83A3A312323A
:1029EB00E1541FF5F0240BF875A025E2FAA312327F
:1029FB00E1541F240BF9E32AF275A025742B25F063
:102A0B00F874FFF2D20F228D828E83A3A31232E1D0
:102A1B00541FF5F0240BF875A025E2FAA31232E14E
:102A2B00541F240BF9E3CAC39AF275A025742B2506
:102A3B00F0F874FFF2D20F228D828E83A3A3123291
:102A4B00E1541FF9903AD87A01122D1F7C10E493B0
:102A5B00FA122D3EA3DCF77AC0122D1F90240074BE
:102A6B0020F0A3F0A3F0A3F0A3E904122C3BEBB4EA
:102A7B0030027420F0A3EAF0A37420F0A3743DF0AD
:102A8B00A37420F0A375A025E9240BF9E3122C3BCA
:102A9B00ECD204B43004C2047420F0A3EBB43005C0
:102AAB002004027420F0A3EAF0A37420F0A3F0A397
:102ABB00F0A3F07C10902400E0FA122D3EA3DCF87A
:102ACB00228D828E83A3A31232E1541FF9FB75A0D2
:102ADB0025240BF9E3FA90001A1232D5C39401B4F2
:102AEB0008005012C423441FF583EB44E0F582EA3F
:102AFB001232C5122CAE228D828E83A3A31232E129
:102B0B00541FF990001A1232D5C39401B408005027
:102B1B0024C423441FF583E944E0F5821232D5FA2D
:102B2B0075A025740B29F8EAF275A025742B29F8EA
:102B3B0074FFF2D20F22C0F08D828E83A3A31232C8
:102B4B00E175F03CA4FEAFF0A31232E1C32EFEEF11
:102B5B003400FFA31232E175F03CFB7C007D00C317
:102B6B00EB2EFBEC3FFCED3400FD15F0E5F070EFC8
:102B7B00A31232E1F879007A009000091232D5B431
:102B8B00000575F0188013B4030575F019800BB4AC
:102B9B00010575F01E800375F01EC3E82BF8E93CA8
:102BAB00F9EA3DFA15F0E5F070F09000091232D514
:102BBB00B4013AEF700BEE6034B40A03022BCC4035
:102BCB0018C3EE940AFEEF9400FFC3E89412F8E9E1
:102BDB009400F9EA9400FA80DAC3EE9401FEC3E89C
:102BEB009402F8E99400F9EA9400FA80C690350053
:102BFB00E0FD903501E0FC903502E0FBC3E89BFF64
:102C0B00E99C7014EA9D701090001B1232D5F5F000
:102C1B00EFB5F002800840069035037401F0903553
:102C2B0000EAF0903501E9F0903502E8F0D0F0229F
:102C3B007A007B007C00601675F00A84AAF0600EA7
:102C4B0075F00A84ABF0600675F00A84ACF0EA24E8
:102C5B0030FAEB2430FBEC2430FC229000001232D3
:102C6B00D5FB9020001232D5FDEBF41232C5122C9D
:102C7B00AE1232D5F4B5030E9000001232D5B50367
:102C8B00057A18022C937A08902000ED1232C512A7
:102C9B002CAE90257FEAF022122C6690257FE0FA6D
:102CAB00F599227C0075F032DCFED5F0FB227A80A0
:102CBB00122D1F7B28902580122D60F0A3DBF97A53
:102CCB00C0122D1F7B28122D60F0A3DBF9227A8016
:102CDB00122D1F7B28902580E0FA122D3EA3DBF8E6
:102CEB007AC0122D1F7B28E0FA122D3EA3DBF822AF
:102CFB007A80122D1F7400936007FA122D3EA38069
:102D0B00F4227AC0122D1F7400936007FA122D3E25
:102D1B00A380F422C0F030111775F00075A09878DD
:102D2B0002E230E70700D5F0F3022D3B7800EAF220
:102D3B00D0F022C0F030111A75F00075A09878020F
:102D4B00E230E70700D5F0F3022D5D75A09878010E
:102D5B00EAF2D0F022C0F030111975F00075A0988E
:102D6B007802E230E70700D5F0F3022D7E75A098CC
:102D7B007803E2D0F02275A0707800EAF4F22222F8
:102D8B00AE82AF83902200EA2323232582F582743F
:102D9B00003583F583E0F8A3E0F9EA245DF5A0891B
:102DAB00F08E828F831232E1F2A308E8B5F00302B2
:102DBB002DFFDBF1AE82AF83902200EA2323232584
:102DCB0082F58274003583F583E8BA000FC2ACF04C
:102DDB00200804D208D299D2AC022DF9D20BF09074
:102DEB002064EA14540F2582F582E0D2E7F0E48EDA
:102DFB00828F832274FF8E828F8322AE82AF839069
:102E0B002200EA2323232582F58274003583F58380
:102E1B00E0F8A3E0F9EA245DF5A089F08E828F83B8
:102E2B001232E1B4F308DB1C0BA3E8022EB9B4F4A5
:102E3B0008DB330BA3E8022EB9B4F56EDB4A0BA308
:102E4B00E8022EB9A31232E1B4F303022EB514A398
:102E5B00C082C08390250B2582F582E0D083D0827F
:102E6B00122F0F022EB9A31232E1B4F403022EB5C6
:102E7B0014A3C082C08390250B2582F582E0D083FA
:102E8B00D082122F60022EB9A31232E1B4F50302E5
:102E9B002EB514A3C082C08390250B2582F582E04A
:102EAB00D083D082122F0B022EB9122F0BA3B5F0A9
:102EBB0006022F04022E2BDBFBAE82AF8390220087
:102ECB00EA2323232582F58274003583F583E8BA40
:102EDB00000FC2ACF0200804D208D299D2AC022E5B
:102EEB00FED20BF0902064EA14540F2582F582E099
:102EFB00D2E7F0E48E828F832274FF8E828F83223F
:102F0B00F208E8227F017E20C39464400C1F7E31BF
:102F1B00C394644004C394640E2464BE2002800EE8
:102F2B00C0E0EE122F0BB5F003022F5FD0E07E3125
:102F3B00C3940A40030E80F81E240AC0E0BE30037F
:102F4B00EF700AEE122F0BB5F003022F5FD0E024C7
:102F5B0030122F0B227F017E30C39464400C1F7EF6
:102F6B0031C394644004C394640E2464C0E0EE1235
:102F7B002F0BB5F003022FADD0E07E31C3940A4086
:102F8B00030E80F81E240AC0E0BE3005EF60027EFF
:102F9B0030EE122F0BB5F003022FADD0E024301220
:102FAB002F0B22200B030230529000121232D5F558
:102FBB00F0A31232D5F58385F082A3E5822411F5B7
:102FCB0082E5833400F583AE82AF8390206475A0D5
:102FDB00887A00C082C0838E828F831232D554E0F0
:102FEB00B4E007D083D08202303AD083D082E03075
:102FFB00E73DC2E7F0EAC4032488F5A07802C0825B
:10300B00C0838E828F831232D5B40A168FF074650B
:10301B00F27FD7C2AFDFFE7475F27F24DFFED2AF33
:10302B00AFF0D083D08274A5F20808087406F2A31F
:10303B00C082C0838E828F83A3AE82AF83D083D0B6
:10304B00820ABA028EC20B228D828E83A3A3123206
:10305B00E114540FC4032488F5A07802A31232E1C3
:10306B00F9C2AF7465F274A5F27FDEE9DFFED9FC1D
:10307B00F97475F27F6FDFFED9FC74B5F2D2AF2213
:10308B0090000A1232D56016758C00758A00D2A991
:10309B00D2AA7530FFF534853433D2078039C20795
:1030AB009000091232D5B4000875366A7535088060
:1030BB001CB401087536877535E98011B4030875A2
:1030CB003670753508800675368875350885368CEB
:1030DB0085358AC2AAD2A9D20222E54E70030231EB
:1030EB0087854E4F7A007B007800792A7D0075F03A
:1030FB002675452075440085458285448312139EB1
:10310B00AE82AF8374052582F58274003583F58317
:10311B007C04C204C2051232D5A36002D20412325F
:10312B00D5A3B4FF028002D205DCEB3004178882F2
:10313B008983EEF0A3EFF0A3E54EC3954FF0A3A365
:10314B00A882A9830B3005198D8285F083EEF0A33D
:10315B00EFF0A3E54EC3954FF0A3A3AD828583F0AB
:10316B000A854582854483A3A3858245858344D5FF
:10317B004F8590257EEBF090257DEAF022C2A87852
:10318B00087A007B029000121232D5F5F0A31232AE
:10319B00D5F58385F082A31232D5F523A3AE82AF8A
:1031AB0083E5822410F582E5833400F5831232D552
:1031BB00FD75A021BD00067400D2E78055BD050644
:1031CB007402D2E7804CBD06067402D2E78043BD81
:1031DB000C067401D2E7803ABDE0067404D2E78096
:1031EB0031BD0D067405D2E78028BD11067409D2D6
:1031FB00E7801FBD0E067407C2E78016BD0F06746D
:10320B0006D2E7800DBD10067408D2E78004740364
:10321B00C2E7F2FCE82402F975A022ECF3BDE0034F
:10322B000232A7EA2488F5A0790009097410F31972
:10323B00197402A21EB392E0BD00028003BD0E04FE
:10324B0044188011A21BB392E4A21C92E2A21D505F
:10325B0004C2E4D2E3F37407301F02740FF3EA24C1
:10326B0088F5A079019032BDE5235407FC93F3EA6E
:10327B002488F5A079047488BC06028008BD050279
:10328B008003BD06027408F3EA2488F5A079027462
:10329B0001F3EA2488F5A079057404F38F838E82F9
:1032AB00E82408F8EA2408FADB0280030231A2D2F0
:1032BB00A82244668899BBCCCCBBC083C0E0E58315
:1032CB0024A0F583D0E0F0D08322C083E58324A033
:1032DB00F583E0D08322300D04E4938011300A0390
:1032EB00E0800BC083E58324A0F583E0D0832274B8
:1032FB00E775F0007F0812331B75F00474007F1024
:10330B0012331B75F00374C07F0F12331BD297223D
:10331B00D295C295C0E07410C39FFE600CD0E03311
:10332B00C5F033C5F0DEF8C0E0D0E0C29020F70462
:10333B00C2978002D297D295C29533C5F033C5F0B0
:10334B00DFEBD290D295C295227A007B32DAFEDB8C
:10335B00FC22300706753000C28C32C0D0C0E0C0F2
:10336B0083C08275D01030071C758C00758A00D213
:10337B008CE40530B530037530FFD5330585343318
:10338B0080030235CDD55003755010E538B40004D9
:10339B00D2B480041538C2B4E537B40004D2B5807A
:1033AB00041537C2B5300005D54102C200E52870BF
:1033BB00030234AF30401B902001E014F07013C2B5
:1033CB0040B220902040E030E008902000E0A3F0D5
:1033DB00D24030411B902003E014F07013C241B275
:1033EB0021902040E030E108902002E0A3F0D24190
:1033FB0030421B902005E014F07013C242B22290B1
:10340B002040E030E208902004E0A3F0D2423043A9
:10341B001B902007E014F07013C243B2239020409E
:10342B00E030E308902006E0A3F0D24330441B9039
:10343B002009E014F07013C244B224902040E03015
:10344B00E408902008E0A3F0D24430451B90200BF9
:10345B00E014F07013C245B225902040E030E5082F
:10346B0090200AE0A3F0D24530461B90200DE014CB
:10347B00F07013C246B226902040E030E608902050
:10348B000CE0A3F0D24630472290200FE014F070EE
:10349B001AC247B227902040E030E70F90200EE091
:1034AB00A3F0D247E52970030235A630481B9020C4
:1034BB0011E014F07013C248B228902041E030E0C4
:1034CB0008902010E0A3F0D24830491B902013E065
:1034DB0014F07013C249B229902041E030E10890FA
:1034EB002012E0A3F0D249304A1B902015E014F0D3
:1034FB007013C24AB22A902041E030E208902014A7
:10350B00E0A3F0D24A304B1B902017E014F070135D
:10351B00C24BB22B902041E030E308902016E0A381
:10352B00F0D24B304C1B902019E014F07013C24CAE
:10353B00B22C902041E030E408902018E0A3F0D2A8
:10354B004C304D1B90201BE014F07013C24DB22D6C
:10355B00902041E030E50890201AE0A3F0D24D30E6
:10356B004E1B90201DE014F07013C24EB22E902013
:10357B0041E030E60890201CE0A3F0D24E304F1B08
:10358B0090201FE014F07013C24FB22F902041E037
:10359B0030E70890201EE0A3F0D24F300211D20189
:1035AB00B294853E83853F82A385833E85823F20EF
:1035BB000710C28CE58A2535F58AE58C3536F58CF6
:1035CB00D28CD082D083D0E0D0D032C0D0C0E0C07B
:1035DB0083C082C01F75D018209811309903023612
:1035EB00AAD01FD082D083D0E0D0D032C298E5874A
:1035FB004440F587309F2AC29F902100E0547FB44E
:10360B0000117401F0E58754BFF587759840D29C83
:10361B0002362C7400F0E58754BFF5877598C0D23D
:10362B009CE58754BFF587902100E0547FB40003DD
:10363B00023653A3E0F58275835AE599F00582E5CE
:10364B0082902101F00236A7902101E0F8A3E0F966
:10365B00A3E0FAA3E0FBE599FF309A1030E70DC227
:10366B009A7B01E8FA0AEA6970027B00EB6021752C
:10367B00835A8A82EFF00582E5826970047B0080B1
:10368B000FAA820B309A098882EB14F0EAF87B00C0
:10369B00902101E8F0A3A3EAF0A3EBF00235E3C21B
:1036AB00991014030236B4A1E3902200E0F8A3E0D2
:1036BB00B5180CE4902203F0A3F0C2080235E39096
:1036CB002100E0547FB40030F8902204E0701275B2
:1036DB00835D8882E0902203F0902201E004F08069
:1036EB0011F8902203E014B5180CE4902203F0A318
:1036FB0014F0D29B8002C29B902201E075835DF592
:10370B0082E0F5990582E582902201F0A3A3A3E064
:10371B0004F00235E3C0D0C0E0C0F0C083C08275B6
:10372B00D018753C02753D00753B00E53B90880554
:10373B002583F583E020E20302380AC0E0902108DC
:10374B00E53B2582F582E0FCA385823A85833954DB
:10375B007FB4000E908801E53B2583F583E0A2E55D
:10376B00920C908803E53B2583F583E0F5F0EC2084
:10377B00E703023808547FB400030237A8853A8266
:10378B00853983E0F582E53D245BF583E5F0F005B3
:10379B0082E582853A82853983F0023808853A8240
:1037AB00853983E0FCA3E0FDA3E0FEA3E0FFE5F099
:1037BB00300C1030E70DC20C7F01ECFE0EEE6D707D
:1037CB00027F00EF60258E82E53D245BF583E5F0FB
:1037DB00F00582E5826D70047F00800FAE820F30A2
:1037EB000C098C82EF14F0EEFC7F00902109E53B75
:1037FB002582F582ECF0A3A3EEF0A3EFF0D0E0204E
:10380B00E003023947902208E53D2323232582F567
:10381B0082E0FFA3E0B51F22A3A37400F0A3F090F6
:10382B008802E53B2583F58374B1F0908805E53B71
:10383B002583F5837404F0023947F5F085823A85C8
:10384B008339A3E0547FB400028008B407028003DD
:10385B00023923C0E0A3E0FC600114FEA3E0FDD01D
:10386B00E0B40705BC00538003BC001FE5F0F582F4
:10387B00E53D245EF583E0FC0582E582853A828591
:10388B003983F0F5F0B51F07023823EDB51E2B90E9
:10389B008802E53B2583F5837415F0908800E53BA2
:1038AB002583F583E0FEA3A37415F0908800E53B18
:1038BB002583F583EE4404F08029908802E53B25AF
:1038CB0083F5837415F0908800E53B2583F583E041
:1038DB00FEA3A37415F0908800E53B2583F583EEDA
:1038EB0054FBF0E5F0F582E53D245EF583E0FE0543
:1038FB0082E582853A82853983F00DECB51D047C17
:10390B00007D00A3A3ECF0A3EDF0908803E53B252D
:10391B0083F583EEF0023947E5F0F582E53D245E51
:10392B00F583E0F5F00582E582853A82853983F0EF
:10393B00908803E53B2583F583E5F0F0053DE53BFA
:10394B002408F53BD53C028003023736D082D08366
:10395B00D0F0D0E0D0D03215F115F1144A14501438
:10396B0056145C146214F814F814F814FB150114B3
:10397B0068147414AA14B014B614C8149E148014CA
:10398B0086148C1498149214CE14D414DA14E014F4
:10399B00F214F814F814F815C715CD1507150D15F5
:1039AB00D915DF14A4147A15131519151F15251520
:1039BB002B1531153715611567156D1573157915A0
:1039CB007F1585158B159115BB15C115D314EC15EA
:1039DB00E51EB41FA0202314E615F1146E14BC14BD
:1039EB00C2153D15431549154F1555155B15971503
:1039FB009D15A315A915AF15B514F814F814F814E3
:103A0B00F814F814F814F814F814F814F814F8144B
:103A1B00F814F814F814F815EB14F815F115F11552
:103A2B00F115F115F115F117536372697074656433
:103A3B002042696E6C6F6F702056362E35300D003C
:103A4B002053637269707465642042696E6C6F6F8A
:103A5B00702076362E353020200020416C636F723B
:103A6B006E204D63427269646520002053686F7746
:103A7B0020646174613A2062616420002053686F96
:103A8B007720646174613A20206F6B200020466CB4
:103A9B0061672042616E6B20232031202020466C11
:103AAB0061672042616E6B20232032202020466C00
:103ABB0061672042616E6B20232033202020466CEF
:103ACB0061672042616E6B20232034202053746188
:103ADB007465205661726961626C65202357616958
:103AEB0074696E6720666F722020202020202020B2
:103AFB0020202020202020202020202020202020BB
:103B0B0020202020200065787465726E616C207314
:103B1B00796E632E2E2E2020202020202020202086
:103B2B002020202020202020202020202020004585
:103B3B00787465726E616C2073796E63202020201F
:103B4B00202020202020202020202020202020206A
:103B5B0020202020202020007265636F766572651F
:103B6B00642E2020202020202020202020202020F8
:103B7B00202020202020202020202020202020203A
:013B8B000039
:00000001FF
